:100000000C942A0B0C94520B0C94520B0C94520B24
:100010000C94520B0C94520B0C94520B0C94520BEC
:100020000C94520B0C94520B0C941C1A0C948E1AB8
:100030000C94520B0C94520B0C94520B0C94520BCC
:100040000C94520B0C94520B0C94520B0C94520BBC
:100050000C94520B0C94520B0C94520B0C94290ED2
:100060000C94520B0C94520B0C94520B0C94520B9C
:100070000C94520B0C94520B0C94520B0C94520B8C
:100080000C94690D0C94520B0C94520B0C94520B63
:100090000C94520B0C94520B0C94520B0C94520B6C
:1000A0000C94520B0C94520B0C94520B99189C18F4
:1000B0008B188F189318BD18BD18BD18A018A41858
:1000C000A818AE18B218BD18B81807634236B79B07
:1000D000D8A71A39685618AEBAAB558C1D3CB7CCA8
:1000E0005763BD6DEDFD753EF6177231BF00000020
:1000F000803F08000000BE922449123EABAAAA2A03
:10010000BECDCCCC4C3E00000080BEABAAAAAA3E1D
:1001100000000000BF000000803F00000000000859
:100120004178D3BB4387D1133D190E3CC3BD4282F6
:10013000AD2B3E68EC8276BED98FE1A93E4C80EFB4
:10014000FFBE01C4FF7F3F0000000000070605045A
:100150000100080A0B0C0D09F0F89C8E8783878E2E
:100160009CF8F00000FEFF0303030303070EFCF8F6
:100170000000FEFF0303030303070EFCF80000FF6B
:10018000FF00000000000000FFFF0000FEFF83836F
:10019000838383C7EE7C380000F8FC0E070303035B
:1001A000070EFCF800003F7FE0C08080C0E07F3F8A
:1001B000FFFF01010101010101FFFF0000FFFF0C32
:1001C0000C0C0C1C3E77E3C100007FFFC0C0C0C018
:1001D000C0E0703F1F00001F3F70E0C0C0C0E07073
:1001E0003F1F00007FFFC1C1C1C1C1E3773E1C00BA
:1001F000001F3F70E0C0C0C0E0703F1F0000000063
:100200000001FFFF01000000D5F08D14A1C881CFCF
:10021000D9F1AF200027253F3F3F253F3F01393F20
:10022000073F3F253D37273D3D1C123F3F31253FCE
:100230003F33392F2F223F3F203F213F3F0E10E019
:10024000FEFEFEFEFFFFFFFFFFFEFEFC3C0303077A
:100250000707070F0F0F0F070703000E10E01E021E
:100260000206050509F9090A06C43C030204040450
:1002700004080F08080404030009081EFEFFFF7F9E
:100280007F7F3F1809081EE68583434F7127180DAD
:100290001010387CFEFFFFFFFFFFFE7C38100000CF
:1002A00000000101010101000000000D10102844B0
:1002B0008201834529119254381000000000010189
:1002C000010101000000001818000080F0F8FCFC9B
:1002D000FEFFFFFFFFFEFEFEFEFCFCFCFCFCF8F850
:1002E0001880F8FFFFFFFFFFFFFFFFFFFFFFFFFF8B
:1002F000FFFFFFFFFFFF1F010003030307070707BF
:10030000070F0F0F0F0F0F1F1F1F0F0F0701000009
:10031000001818000080700804C47EAB55AB55AAC5
:1003200056AA56AC54AC54AC58E81880780780C034
:10033000FCAB55AA55AA55AA55AA55AA55AA55EADD
:100340001F01000303030404040405090909090A41
:100350000B1213120D0E07010000001418C0E0E08C
:10036000F0F8F8FCFCFEFEFEFEFDFFFEFCF0C00017
:100370000000030F3FFFFFFFFFFFFFFFFFFF7F7F37
:100380003F3F1F1F0C0000000000000001010101A1
:100390000000000000000000001418C0606050C899
:1003A00068A454B25AAA56AD57AA5CB0C000000067
:1003B000030C30C0838E35EA55AAD5AA556A352A72
:1003C000151B0C00000000000000010101010000ED
:1003D00000000000000000191800000080E0F8FC98
:1003E000FEFEFEFFFFFFFFFFFEFEFCFCF8F8F0F054
:1003F000E060103C3F7F7FFFFFFFFFFFFFFFFFFF3D
:10040000FFFFFFFFFFFF7F1F07010000000000004C
:1004100000010103030707030303010101000000BA
:1004200000000000191800000080E0F8FCFEFEFA51
:10043000FDFBF5EBF5EAD6ACD4A8587050A06010DF
:100440003C3F7F7FFFFFFFFFFFFFFFFF7F1F070393
:10045000008080601806010000000000000001011B
:10046000030307070202020101010000000000006F
:100470000018180080C0E0F0F8FCFEFFFFFFFFFF4F
:10048000FFFFFFFFFFFFFFFCE08000030F3FFFFFC8
:10049000FFFFFFFFFFFFFFFFFFFFFFFFFFFFFF7FEC
:1004A0003F1F0C00000000030F0F0F0F0F0F0F0F67
:1004B0000F0F0F070301000000000018180080C094
:1004C000E0F0F8FCFEFFFFFFFFFF7FBF5FAF57AB21
:1004D00057BC608000030D31C10101010101010120
:1004E000030E75AA55AA55AAD56A351B0C00000043
:1004F00000030C0808080808080808090F0603018B
:10050000000000000017080103070F1F3F7FFFFFD7
:100510007F7F3F3F1F1F0F0F0707030301011708CE
:100520000102050A152A55AAD56A552A351A150A4F
:100530000D06050203010106080012040812000658
:10054000083F3F3F3F3F3F0608000C12120C0006D9
:10055000081E3F3F3F3F1E3008003E3E0A04001E7B
:100560003E201E002E2E2A3A003E3E083E0000008D
:100570002E2E2A3A00023E3E02003C3E0A3E003E3B
:100580003E0A3400023E3E020030087F7F7F7F1F1C
:100590003F7F7F7F7F7F7F7F7F7F7F7F7F7F7F7FAB
:1005A000007F7F7F7F7F7F7F7F7F7F7F7F7F7F7FDA
:1005B0007F7F7F7F7F7F7F7F7F7F07201800FC0208
:1005C000BADA0AFAFA0ADABA02FA027A4A7AB2020B
:1005D000FAF20A52BA6AE2CA9A3A02FC00000F1012
:1005E0001717141317101717E007F8F7F6B55BF88D
:1005F00003E71017161512151713140F000000004B
:1006000000000000000000003F40574B554A554B8A
:10061000403F00000000000000000000002018FE25
:10062000FFFFFFFFFFFFFFFFFFFFFFFFFFFFFFFFDA
:10063000FFFFFFFFFFFFFFFFFFFFFFFFFFFFFE1FAB
:100640003F3F3F3F3F3F3F3F3FFFFFFFFFFFFFFF7A
:10065000FFFFFFFFFF3F3F3F3F3F3F3F3F3F1F0049
:10066000000000000000000000FFFFFFFFFFFFFF91
:10067000FFFFFFFFFF000000000000000000000679
:10068000080018003C7E0006083C3C7EFFFFFF0887
:100690000855A0548055A0548054314F3442310045
:1006A0001010F0F0F0F0FFFFFFFFF0F0F0F00000AE
:1006B000000000000000000000000000000000003A
:1006C000000000000000FFFFFFFFF0F0F0F000006E
:1006D0000000000000000F0F0F0F000000000000DE
:1006E0000000F0F0F0F0F0F0F0F0F0F0F0F00000CA
:1006F0000000000000000F0F0F0F000000000000BE
:100700000000F0F0F0F0FFFFFFFF0000000000002D
:100710000000000000000F0F0F0F0000000000009D
:100720000000101000606060607E7E6060606000AD
:1007300000000000000000000000000000000000B9
:10074000000000000000000000FEFE60606060002D
:10075000000000000000000000070700000000008B
:10076000000000000060606060E0E06060606000C9
:10077000000000000000000000070700000000006B
:10078000000000000060606060FEFE0000000000ED
:10079000000000000000000000070700000000004B
:1007A00000000000101000000000F0F0F0F0F0F089
:1007B000F0F0000000000F0F0F0F0F0F0F0F0000E1
:1007C00000000000000000000000FFFFFFFFF0F04D
:1007D000F0F00000000000000000000000000F0F1B
:1007E0000F0F000000000000000000000000F0F00B
:1007F000F0F0F0F0F0F0000000000F0F0F0F0F0FFF
:100800000F0F0000000000000000F0F0F0F000000A
:10081000000000000000000000000F0F0F0FFFFF9E
:10082000FFFF0000000010100000000000A04020AA
:100830004020400000000000000204020402050005
:1008400000000000000000000000000000542A40EA
:100850002040A00000000000000000000000000098
:100860000005020000000000000000000000000081
:1008700000A04020402040000000000000020402D0
:100880000402050000000000000000000040A0007D
:10089000000000000000000000000000000502044D
:1008A00002542A0000000000101000000000F0F0C8
:1008B000F0F0F0F0F0F00000000000000000000098
:1008C00000000F0F0F0F0F0F0F0F000000000000B0
:1008D0000000F0F0F0F00000000000000000FFFF5A
:1008E000FFFF0F0F0F0F00000000F0F0F0F0F0F02E
:1008F000F0F00000000000000000000000000F0FFA
:100900000F0F0F0F0F0F0000000000000000F0F0AD
:10091000F0F0FFFFFFFF00000000000000000F0FDD
:100920000F0F000000000000000010100000000089
:100930000020402040A04000000000000000000017
:100940000000000000020502040204000000000094
:10095000000000000040A0000000000000000000B7
:1009600000542A040205020000000000002040207C
:1009700040A0400000000000000000000000000057
:100980000002050204020400000000000000000054
:100990000040A04020542A00000000000000000099
:1009A0000005020000000000000000001010000020
:1009B0000000F0F0F0F0F0F0F0F0000000000000B7
:1009C00000000F0F0F0F0F0F0F0F000000000000AF
:1009D0000000F0F0F0F0F0F0F0F000000000000097
:1009E00000000F0F0F0F0F0F0F0F0000000000008F
:1009F0000000F0F0F0F0F0F0F0F000000000000077
:100A000000000F0F0F0F0F0F0F0F0000000000006E
:100A10000000F0F0F0F0F0F0F0F000000000000056
:100A200000000F0F0F0F0F0F0F0F0000000010102E
:100A30000000000000E020202020E0000000000076
:100A40000000000000070404040407000000000088
:100A50000000000000E020202020E0000000000056
:100A60000000000000070404040407000000000068
:100A70000000000000E020202020E0000000000036
:100A80000000000000070404040407000000000048
:100A90000000000000E020202020E0000000000016
:100AA0000000000000070404040407000000000028
:100AB0001010F0F0F0F0F0F0F0F0F0F0F0F00000D6
:100AC000000000000000000000000F0F0F0F0000EA
:100AD00000000000000000000000FFFFFFFF00001A
:100AE0000000000000000F0F0F0F0F0F0F0F00008E
:100AF000000000000000F0F0F0F000000000000036
:100B00000000000000000F0F0F0F0F0F0F0F0F0F4F
:100B10000F0F00000000F0F0F0F0F0F0F0F0000037
:100B2000000000000000FFFFFFFF000000000000C9
:100B300000001010006020406020406020C0600075
:100B4000000000000000000000000000000603009C
:100B500000000000000000000000000000DAB60005
:100B6000000000000000000000020604020605006C
:100B7000000000000000000000C060000000000055
:100B80000000000000000000000603040602040646
:100B9000020406000000000000A060402060400049
:100BA0000000000000000000006D5B00000000007D
:100BB00000000000101000000000F0F0F0F0F0F075
:100BC000F0F0F0F0F0F0000000000F0F0F0F000049
:100BD00000000000000000000000F0F0F0F0F0F075
:100BE000F0F0000000000000000000000000FFFF27
:100BF000FFFF000000000000000000000000F0F017
:100C0000F0F0000000000F0F0F0F0F0F0F0F0F0F6E
:100C10000F0F0000000000000000FFFFFFFF0000BA
:100C2000000000000000000000000F0F0F0F0F0F6A
:100C30000F0F000000001010000000000060A04036
:100C400060204060204060000000000000030500BC
:100C500000000000000000000000000000402060D4
:100C600040A0600000000000000000000000000044
:100C7000006D5B00000000000000000000000000AC
:100C800000A0C000000000000006020406020406E6
:100C900002050600000000000000000000DAB600B7
:100CA0000000000000000000000000000006050237
:100CB00006040200000000001010F0F0F0F0F0F068
:100CC000F0F0F0F0F0F0F0F0F0F0000000000000C4
:100CD0000000000000000000000000000000000014
:100CE0000000FFFFFFFF0000000000000000000008
:100CF0000000FFFFFFFF00000000000000000000F8
:100D0000000000000000000000000F0F0F0F0F0F89
:100D10000F0F0F0F0F0F0F0F0F0F00000000FFFF3F
:100D2000FFFF000000000000000000000000FFFFC7
:100D3000FFFF000000000000000010100060606075
:100D40006060606060606060606060000000000083
:100D50000000000000000000000000000000000093
:100D60000000000000FEFE00000000000000000087
:100D700000000000007F7F00000000000000000075
:100D80000000000000000000000000000006060651
:100D90000606060606060606060606000000000011
:100DA00000FEFE0000000000000000000000000047
:100DB000007F7F0000000000000000001610001CF3
:100DC0003E223A003C3E0A3E003E3E1C0C3E003EA7
:100DD0003E2A220000387C444438003C7C403C00E1
:100DE0007C7C5444007C7C14680016103E7F7F7F1E
:100DF0007F7F7F7F7F7F7F7F7F7F7F7F7F7F7F7F03
:100E00007F777CFEFEFEFEFEFEFEFEFEFEFEFEFE8A
:100E1000FEFEFEFEFEFEFEFE0F090D0F0F0808008F
:100E20000F000F02040F000F0B09000B0D0D0F0236
:100E3000040F000F0B090009060900010F010F083C
:100E4000000F0B0900070807000F0B09000F080B24
:100E50000D000F0900060906000F050A000F0B0917
:100E600054A854A854A850AE5602FEFE02A64E0046
:100E7000FE00DE925EAC00FEFC00D4AE5AB872E614
:100E8000CE2054A854A854A854000000000000002C
:100E9000000000000100000000010001010100004D
:100EA000000100010101000101000000000000003C
:100EB000000000000000010101010000000000002E
:100EC000000000000100000001000000010000001F
:100ED000010000000000000000000101010100000D
:100EE00000000001000000010000000100000001FE
:100EF00000000000000000010101000100000000EE
:100F000000000000000000010100000001000000DE
:100F100001000000000000000100010101000000CC
:100F200000000001000000010000000101000000BD
:100F300000000000000001010100000001000000AD
:100F4000000000000100000001000001010000009D
:100F5000000000000000000100000001010100008D
:100F6000000000000000000101000001000000017D
:100F7000000000000000000101000001010000006D
:100F8000000000000000000101000001010000005D
:100F9000000000000000000101000001010000004D
:100FA000000000000000000101000001010000003D
:100FB000000000000000000101000000010100002D
:100FC000000000000000000001000001010000011D
:100FD000000000000000010100000001010000000D
:100FE00000000000010000010100000100000000FD
:100FF00000000000000000010100010100000000ED
:1010000000000001000000010100000001000000DC
:1010100000000000000000000101000101000000CC
:1010200000000000000000010000000101000000BD
:1010300001000001000001010100000000000000AB
:10104000000000010000000101000001000000009C
:10105000000000000000010101000001000000008C
:10106000000000010000010100000001000000007C
:101070000000010204081020408000000000003E33
:101080005B4F5B3E3E6B4F6B3E1C3E7C3E1C183CF8
:101090007E3C181C577D571C1C5E7F5E1C00183C54
:1010A0001800FFE7C3E7FF0018241800FFE7DBE79D
:1010B000FF30483A060E2629792926407F05050784
:1010C000407F05253F5A3CE73C5A7F3E1C1C0808E0
:1010D0001C1C3E7F14227F22145F5F005F5F0609A5
:1010E0007F017F006689956A606060606094A2FFFE
:1010F000A29408047E040810207E201008082A1CF0
:1011000008081C2A08081E101010100C1E0C1E0CBB
:1011100030383E3830060E3E0E060000000000005B
:10112000005F00000007000700147F147F14242ACA
:101130007F2A12231308646236495620500008079C
:101140000300001C2241000041221C002A1C7F1CBD
:101150002A08083E080800807030000808080808BF
:10116000000060600020100804023E5149453E0026
:10117000427F400072494949462141494D33181484
:10118000127F1027454545393C4A494931412111D3
:1011900009073649494936464949291E00001400C5
:1011A00000004034000000081422411414141414E8
:1011B000004122140802015909063E415D594E7C46
:1011C0001211127C7F494949363E414141227F41FB
:1011D00041413E7F494949417F090909013E414159
:1011E00051737F0808087F00417F41002040413F44
:1011F000017F081422417F404040407F021C027F53
:101200007F0408107F3E4141413E7F090909063EA7
:101210004151215E7F091929462649494932030176
:101220007F01033F4040403F1F2040201F3F403888
:10123000403F631408146303047804036159494D63
:1012400043007F4141410204081020004141417F99
:10125000040201020440404040400003070800200F
:10126000545478407F28444438384444442838440F
:1012700044287F385454541800087E090218A4A446
:101280009C787F0804047800447D40002040403D65
:10129000007F1028440000417F40007C04780478DF
:1012A0007C080404783844444438FC182424181872
:1012B000242418FC7C0804040848545454240404CE
:1012C0003F44243C4040207C1C2040201C3C4030BB
:1012D000403C44281028444C9090907C4464544CEA
:1012E0004400083641000000770000004136080045
:1012F00002010204023C2623263C1EA1A161123AEF
:101300004040207A3854545559215555794121543B
:10131000547841215554784020545579400C1E5240
:1013200072123955555559395454545939555454E4
:10133000580000457C410002457D420001457C404B
:10134000F0292429F0F0282528F07C545545002068
:1013500054547C547C0A097F493249494932324805
:10136000484832324A4848303A4141217A3A42406C
:101370002078009DA0A07D39444444393D40404040
:101380003D3C24FF2424487E4943662B2FFC2F2B11
:10139000FF0929F620C0887E0903205454794100B2
:1013A00000447D413048484A32384040227A007A31
:1013B0000A0A727D0D19317D2629292F282629290F
:1013C000292630484D402038080808080808080831
:1013D000382F10C8ACBA2F102834FA00007B000058
:1013E00008142A142222142A14089500220095AA0F
:1013F000005500AAAA55AA55AA000000FF00101027
:1014000010FF00141414FF001010FF00FF1010F064
:1014100010F0141414FC001414F700FF0000FF0077
:10142000FF1414F404FC141417101F10101F101FC5
:101430001414141F00101010F0000000001F1010F2
:1014400010101F10101010F010000000FF101010EE
:10145000101010101010FF10000000FF140000FF0B
:1014600000FF00001F10170000FC04F414141710F4
:10147000171414F404F40000FF00F71414141414E7
:101480001414F700F7141414171410101F101F145D
:101490001414F4141010F010F000001F101F0000BE
:1014A000001F14000000FC140000F010F01010FFEA
:1014B00010FF141414FF141010101F00000000F08F
:1014C00010FFFFFFFFFFF0F0F0F0F0FFFFFF000064
:1014D000000000FFFF0F0F0F0F0F38444438447C0B
:1014E0002A2A3E147E02020606027E027E0263550E
:1014F0004941633844443C04407E201E2006027E5D
:10150000020299A5E7A5991C2A492A1C4C7201726E
:101510004C304A4D4D303048784830BC625A463DD8
:101520003E494949007E0101017E2A2A2A2A2A448D
:10153000445F444440514A444040444A51400000C2
:10154000FF0103E080FF000008086B6B08361236CD
:101550002436060F090F06000018180000001010AE
:10156000003040FF0101001F01011E00191D17126C
:10157000003C3C3C3C000000000000000000250056
:1015800028002B002E003100040404040403040589
:101590000202020204030202020206060606060610
:1015A00004040202020404040802011040804010F6
:1015B0002040804080080204018040201002011079
:1015C0008010204040200000000200090F000003AE
:1015D0000401000C000000000000000000000000FA
:1015E000000000000003080B0002020201000904D1
:1015F0000000010202000005240010010524010181
:1016000001042402060524060001070581031000D9
:101610004009040100020A00000007050202400020
:1016200000070583024000000403090412010002C0
:10163000EF020140412336800001010203014172A3
:101640006475696E6F204C4C430041726475626F23
:101650007900E22411241FBECFEFDAE0DEBFCDBF58
:1016600011E0A0E0B1E0E2E5F4E502C005900D92E2
:10167000A833B107D9F727E0A8E3B1E001C01D9274
:10168000A13AB207E1F71BE0CAE2DBE004C0219710
:10169000FE010E941C2AC932D107C9F70E94BE1C54
:1016A0000C94272A0C940000CF92DF92EF92FF92C5
:1016B0000F931F93CF93DF936C017A018B01C0E0EE
:1016C000D0E0CE15DF0589F0D8016D918D01D601EE
:1016D000ED91FC910190F081E02DC6010995892BD7
:1016E00011F47E0102C02196ECCFC701DF91CF91AA
:1016F0001F910F91FF90EF90DF90CF9008954F9240
:101700005F926F927F928F929F92AF92BF92CF9291
:10171000DF92EF92FF920F931F93CF93DF9300D04E
:1017200000D0CDB7DEB749012C2DA02EB12CDC01A5
:10173000AA0DBB1D1A161B060CF0B3C1803891050B
:101740000CF0AFC1FB01EE0DF11D1E161F060CF0D3
:10175000A8C1603471050CF0A4C14115510509F40C
:10176000A0C1FB0177FF04C0EE27FF27E61BF70BA4
:101770003E2F3770732EFB0177FD379633E0F595DA
:10178000E7953A95E1F73E2F77FF07C0772029F0DC
:101790003FEF3E0F68E06719762E97FF05C0EE27F2
:1017A000FF27E81BF90B02C0E0E0F0E0A038B1052C
:1017B00024F060E8F62EF81A01C0F02EFE1A632F0E
:1017C000032E000C770B3F3F1CF4A62FA09501C001
:1017D000A0E011E0BE2DB77009F410E0E694E694A5
:1017E000E694E10E6E0D711D693071051CF068E024
:1017F000E62EE31AEA1A3A0F60E83603800D911DCF
:1018000011248E0F9F1FA09FE00DF11D11244E0F7C
:101810005F1F61E070E0072C02C0660F771F0A941B
:10182000E2F7233009F4FCC098F4213009F4AEC08B
:10183000223009F036C12FEF269F8001279F100D1F
:101840001124009510951C830B835C80E30E27C048
:101850002A3F29F02B3F09F024C1E30E83C0E30E99
:101860004EC0FA01EC0DFD1DE491E69F4001E79F9B
:10187000900C11249A82898237FD04C02C91202378
:10188000822A8C92711014C0EFEFCE1ADE0A1196E4
:10189000CF1438F33F5F4A0D5B1D80589F4F3E15B4
:1018A00009F4FFC0DC01AF5DBC4FC12CD12CF0CFDF
:1018B000373054F7FD01E058FF4F208125219A80F1
:1018C00029292083E1CFFA01E00FF11FE491E69F7F
:1018D0006001E79FD00C1124DA82C98237FD03C072
:1018E0002C91C22ACC92711013C00F5F1F4F11961A
:1018F0000F1548F33F5F4A0D5B1D80589F4F3E1503
:1019000009F4CFC0DC01AF5DBC4F00E010E0F0CFC8
:1019100037305CF7FD01E058FF4FD0802A812D2938
:101920002083E3CFFA01EC0DFD1DE491E69FD00189
:10193000E79FB00D1124BA83A98337FD05C0A09598
:10194000F8012081A223A083711015C0FFEFCF1AE8
:10195000DF0A0F5F1F4FCF1428F33F5F4A0D5B1D57
:1019600080589F4F3E1509F49CC08C010F5D1C4FA1
:10197000C12CD12CF0CF37304CF7F801E058FF4F95
:101980002A812095A0812A232083E0CFD401AE0FA5
:10199000BF1FE30E3E1509F484C0FC01EF5DFC4F50
:1019A0004F01C12CD12CCF1498F5FD01EC0DFD1D7C
:1019B000E491E69F8001E79F100D1124009510959A
:1019C0001C830B83FA01EC0DFD1DE491E69F2001C1
:1019D000E79F500C11245A82498237FD05C0F4015B
:1019E00020810223402A4082772059F037304CF47E
:1019F000F401E058FF4F10812C8121231A81212B03
:101A00002083FFEFCF1ADF0A2FEF821A920ACBCF83
:101A10003F5F4A0D5B1DAA0DBB1D80589F4FBACF7B
:101A2000CF2CD12CE40FF51FDC01AF5DBC4FAC0116
:101A30004F555C4F00E810E00C191D09AC18BD08AB
:101A4000AA0CBB1C6F2C2E2DCF93DF93EA0185903F
:101A5000C590772059F0869E4001C69E60013730C0
:101A60002CF49881D0949D219929999333233AF0AD
:101A70009C91C0949C2198299D930C94400D1196A3
:101A8000FA9429F7EA9451F0F62C33951124EA0DD3
:101A9000F11DA00FB11DC00FD11DD9CFDF91CF9186
:101AA00011240F900F900F900F90DF91CF911F9105
:101AB0000F91FF90EF90DF90CF90BF90AF909F90ED
:101AC0008F907F906F905F904F90089508950E943F
:101AD000222A1F920F920FB60F9211242F933F9339
:101AE0008F939F93AF93BF93EF93FF9380911903CD
:101AF00090911A03A0911B03B0911C03E09116036F
:101B0000F0911703892B8A2B8B2B31F180911803CD
:101B10009081892780838091190390911A03A09165
:101B20001B03B0911C03181619061A061B062CF588
:101B30008091190390911A03A0911B03B0911C038B
:101B40000197A109B1098093190390931A03A093F7
:101B50001B03B0931C0311C0809171008D7F809393
:101B60007100909118038081282F30E0892F90E038
:101B700080959095822393238083FF91EF91BF916D
:101B8000AF919F918F913F912F910F900FBE0F902A
:101B90001F9018953FB7F89480911203909113030A
:101BA000A0911403B091150326B5A89B05C02F3F43
:101BB00019F00196A11DB11D3FBFBA2FA92F982F73
:101BC0008827820F911DA11DB11DBC01CD0142E0EE
:101BD000660F771F881F991F4A95D1F708958F9236
:101BE0009F92AF92BF92CF92DF92EF92FF926B01E2
:101BF0007C010E94CA0D4B015C01C114D104E104B7
:101C0000F104F1F00E94CA0DDC01CB018819990999
:101C1000AA09BB09883E9340A105B10570F321E0F4
:101C2000C21AD108E108F10888EE880E83E0981EF8
:101C3000A11CB11CC114D104E104F10419F7DDCFDA
:101C4000FF90EF90DF90CF90BF90AF909F908F90DC
:101C500008951F920F920FB60F9211242F933F9366
:101C60008F939F93AF93BF9380914C0190914D01BF
:101C7000A0914E01B0914F013091110323E0230F49
:101C80002D3720F40196A11DB11D05C026E8230FB4
:101C90000296A11DB11D2093110380934C019093D6
:101CA0004D01A0934E01B0934F018091120390918A
:101CB0001303A0911403B09115030196A11DB11D4A
:101CC0008093120390931303A0931403B09315030E
:101CD000BF91AF919F918F913F912F910F900FBE28
:101CE0000F901F901895CF92DF92EF920F93CF93A2
:101CF000DF934115510569F1FA0104913196E490A1
:101D00004E5F5F4F2223F9F0C02FD0E0AE2DA69595
:101D1000A695A695EA2FF0E0A1E0B0E03E2D377041
:101D200011F4A0E0B0E0AE0FBF1FCA9F6001CB9FCF
:101D3000D00CDA9FD00C11242C9DF0012D9DF00DBC
:101D400011244E0F5F1F2AEFC22E20E030E00E94C8
:101D50007F0BDF91CF910F91EF90DF90CF9008959F
:101D6000CF92DF92EF920F93CF93DF9341155105FE
:101D700069F1FA0104913196E4904E5F5F4F22239E
:101D8000F9F0C02FD0E0AE2DA695A695A695EA2F26
:101D9000F0E0A1E0B0E03E2D377011F4A0E0B0E03B
:101DA000AE0FBF1FCA9F6001CB9FD00CDA9FD00C33
:101DB00011242C9DF0012D9DF00D11244E0F5F1F5D
:101DC0002BEFC22E20E030E00E947F0BDF91CF91FD
:101DD0000F91EF90DF90CF9008952D9A0895BC0158
:101DE00080E090E00C94EF0D8FB12CB193B130E016
:101DF0002095309520743327A90123E05595479508
:101E00002A95E1F7292F30E020953095207133276E
:101E10003595279535952795242B8095807F822BA6
:101E2000089583B7817F83BF83B7816083BF88951F
:101E300083B78E7F83BF08958EBD00000DB407FE6B
:101E4000FDCF0895109250013E983F9808953E9A14
:101E50003F9A81E08093500108952F923F924F92D4
:101E60005F926F927F928F929F92AF92BF92CF922A
:101E7000DF92EF92FF920F931F93CF93DF93CDB733
:101E8000DEB72D970FB6F894DEBF0FBECDBFED8243
:101E9000E22EF12C9C012E0D3F1D37FD32C1803802
:101EA00091050CF02EC19B01200F311D37FD29C17A
:101EB000603471050CF025C1DB0177FF04C0AA274F
:101EC000BB27A61BB70BA770BB279B0177FF02C0E0
:101ED000295F3F4F13E0359527951A95E1F777FF76
:101EE00008C02150310968E070E0FB01EA1BFB0BE0
:101EF000DF01E02FE695E695E695CE2ED12C077012
:101F000019F0FFEFCF1ADF0AB9017695762F662711
:101F100077956795680F791F6F5D7C4F8601020F7B
:101F2000131F19870887C12CD12CF8E0AF2EB12CD4
:101F300085010A1B1B0B1F830E830885198520173B
:101F4000310709F4DEC02830310509F4DAC02F3F2B
:101F50001FEF31070CF4CAC08B0100581F4F1D87BB
:101F60000C874B013B012B011C011C830B831A8343
:101F700009831B861A860A851B850E151F050CF022
:101F8000B5C010E82116310409F4B0C037FC89C08F
:101F90002F3FEFEF3E0709F4B0C00A851B850C0DFB
:101FA0001D1DFD81F13079F4F801E40FF51FE49176
:101FB000F0E08F010A2E01C0000F0A94EAF7F30146
:101FC000B0800B2925C0FD81F11114C0F801E40F88
:101FD000F51FE491F0E00A2E02C0EE0FFF1F0A94F5
:101FE000E2F78F0100951095F401A080B12C0A2131
:101FF0001B210EC0F801E40FF51FE491F0E08F0102
:102000000A2E01C0000F0A94EAF7F201B0800B25F6
:102010000083109709F445C02730310509F441C009
:102020000A851B850C0D1D1DFD81F13089F4F80119
:10203000E40FF51FE4910E2F10E00E8002C01595FD
:1020400007950A94E2F7EC85FD85B0800B2928C03E
:10205000FD81F11115C0F801E40FF51FE4910E2F79
:1020600010E00E8002C0159507950A94E2F70095DE
:102070001095E981FA81A080B12C0A211B2110C0A2
:10208000F801E40FF51FE4910E2F10E00E8002C05E
:10209000159507950A94E2F7EB81FC81B0800B253A
:1020A00000830A851B850F5F1F4F1B870A870C85DE
:1020B0001D850F5F1F4F1D870C8709811A810F5FD8
:1020C0001F4F1A8309830B811C810F5F1F4F1C83D5
:1020D0000B831FEF211A310AEFEF4E1A5E0AFFEF52
:1020E0006F1A7F0A0FEF801A900A45CF2F5F3F4F7C
:1020F00060587F4FCE0CDF1C20CF109709F090CF97
:10210000D0CF2D960FB6F894DEBF0FBECDBFDF91B6
:10211000CF911F910F91FF90EF90DF90CF90BF90E4
:10212000AF909F908F907F906F905F904F903F9077
:102130002F90089560387105D0F440345105B8F4FB
:10214000E2E7F0E180E1849FD001A0781124A60F9E
:102150004770E40FF11DE491AF5DBC4F222319F0ED
:102160004C91E42B03C0E0954C91E423EC9308954B
:102170002F923F924F925F926F927F928F929F9297
:10218000AF92BF92CF92DF92EF92FF920F931F9385
:10219000CF93DF93CDB7DEB729970FB6F894DEBFA4
:1021A0000FBECDBFFC016A3069F4248D808D918D06
:1021B00038E0239F800D911D1124918F808F178A05
:1021C000168AAAC06D3009F4A7C099878887F48C55
:1021D000338C228C608C718C06891789003811052C
:1021E000C4F0A885B9855C962C915C97422F50E08D
:1021F00056968D919C915797B6E02B9F800D911D1F
:102200001124E885F985978B868B258D21116EC069
:1022100083C0F0E46F16710424F7C80125E0F29E34
:10222000800D911D112418161906DCF68F2D90E0F3
:102230009C838B83C301A8E0FA9E800D911D11241D
:102240001816190674F6B5E06B9FB0011124FB0156
:10225000E658FF4EFA83E98330E088859985049635
:102260009E838D83E981FA81E490353009F4E12C75
:10227000430188E0482EE0FC02C0532C01C0522CE0
:1022800051100BC0321009C0E6944A948B819C8196
:10229000880E991E4110EFCF1BC068018C2D801B4A
:1022A0008F1590F754018A2D88198F1568F4252D04
:1022B000A501B6018D819E813F830E949A109FEFF8
:1022C000A91AB90A3F81EFCFAFEFCA1ADA0AE6CFEF
:1022D0003F5FEB81FC810E0F1F1F89819A81019660
:1022E0009A838983363009F0BDCF7BCF6AEF6403D0
:1022F0009001659F300D112420583F4F2817390752
:102300005CF4A885B985ED91FC9111970190F0815D
:10231000E02D6AE0CD01099581E090E029960FB6A5
:10232000F894DEBF0FBECDBFDF91CF911F910F910B
:10233000FF90EF90DF90CF90BF90AF909F908F90E5
:102340007F906F905F904F903F902F9008955F9295
:102350006F927F928F929F92AF92BF92CF92DF92B5
:10236000EF92FF920F931F93CF93DF93C82EC62F48
:102370004A01522E4115510561F4409138015091A6
:10238000390170E0E22E06E024E090E00E942D0F7B
:1023900045C0BA01F12C2AE030E0CB01B9010E941E
:1023A000082AF39461157105C1F7A12CB12C10E036
:1023B0009AE0692E712CD0E0D12C1F1579F1612F94
:1023C00070E080E090E00E945F269B01AC0160E03D
:1023D00070E080E291E40E941D270E943026AB014C
:1023E000BC01C401BA010E94082ACB01B3010E94BA
:1023F000082AFC01EE0FFF1FE85CFE4F408151816F
:10240000E52C06E024E0BE01C5018C0D9D1D0E9457
:102410002D0F1F5F85E0A81AB108CFCFDF91CF91B4
:102420001F910F91FF90EF90DF90CF90BF90AF90F2
:102430009F908F907F906F905F9008950F931F9360
:10244000CF93DF9390919101890F84301CF010920B
:10245000910104C087FD83E08093910180919001F8
:102460002091910161E073E042E551E0A0E034E0A9
:10247000839FC0011124820F911D27FD9A9524E0AE
:10248000880F991F2A95E1F7B1E020E030E0EA2FAC
:10249000E20FEC01CE0FD11DFE01EE54F14FE4919D
:1024A0008B01020F131FEA01C20FD31FEE2321F08D
:1024B000F801B083B88303C0F801108218822F5F3F
:1024C0003F4F2430310519F76C5F7F4F4C5F5F4FF2
:1024D000AC5FA031D1F6DF91CF911F910F9108959C
:1024E00080E090E0DC01AE5ABE4FFC01EF5FFC4F94
:1024F0002C91208311962C911197218312962C9167
:102500001297228313962C91238304968031910590
:1025100049F7089590919101890F843024F487FF41
:1025200003C083E001C080E02091900161E073E08E
:1025300040E0082E000C990B34E0239F800D911D84
:10254000112424E0880F991F2A95E1F751E020E03B
:1025500030E0E42FE20FDC01AE0FB11DFD01EE54BF
:10256000F14FE491DB01A20FB31FEE2311F05C9356
:1025700001C01C922F5F3F4F2430310551F76C5F33
:102580007F4F4C5F403119F708954F925F926F92E1
:102590007F928F929F92BF92CF92DF92EF92FF92A3
:1025A0000F931F93CF93DF93C62FE0906401F82E13
:1025B000FE0C8091650187FD8D5F682F659565959F
:1025C000062E000C770B880B990B0E9461260E9447
:1025D0009C260E942926BC2EB60EEB2D0B2C000C3F
:1025E000FF0BA1E0B3E08F2C0F2C000C99086401C5
:1025F0002B2D3EE02302C00CD11C112440E050E002
:102600002F013A016C0C7D1C20E030E08D01020F9F
:10261000131FE8011881112311F18901060D171DFF
:102620000E561E4FE8011A81112321F0D1E0BD1290
:1026300025C00AC08901080D191D0A301105B0F71F
:10264000E231F10564F0F2CFFE1018C0E201C61BC2
:10265000D70B219799F480E3809391020FC02F5FED
:102660003F4F2430310591F631961496425F5F4F0B
:102670004833510531F681E090E002C080E090E0FF
:10268000DF91CF911F910F91FF90EF90DF90CF904E
:10269000BF909F908F907F906F905F904F90089524
:1026A0000F931F93CF93DF938091510180939001FB
:1026B0000E94A22527E030E040E050E00E94C625BD
:1026C00060935101A091900162E571E041E053E017
:1026D00020E080E4A89FD001112431E080E090E068
:1026E000E22FE80FED01CE0FD11DFE01EE54F14FA8
:1026F000E4918B01080F191FEA01C80FD91FEE23BF
:1027000021F0F8013083388303C0F8011082188269
:1027100001968430910521F76C5F7F4F4C5F5F4FCE
:102720002C5F2031D9F683E080936401109265011B
:1027300010929101DF91CF911F910F910895EF9227
:102740000F93CF93DF93EE24E3940AE029E240E66F
:102750005EE06FE170E080E090E00E942D0FCCE23F
:10276000D0E021E040E460E070E0CE010E94291654
:102770002196C435D105A9F72FE330E04AE250E0B5
:1027800060E070E08AE290E00E94A8172FE330E05A
:1027900045E550E060E070E085E590E00E94A81714
:1027A0004AE063E070E088E090E00E94661748E04D
:1027B00064E070E089E090E00E941017E12C04E0F2
:1027C00021E14FE45EE066E070E08CE090E00E9482
:1027D0002D0FC0E0D0E021E048E063E170E0CE01E1
:1027E0000E9429162196C932D105A9F721E130E0CE
:1027F00048E250E061E170E080E090E00E94A817BC
:102800002CE130E048E250E06CE170E080E090E0E4
:102810000E94A81741E16CE270E087E090E00E941E
:1028200066174FE06DE270E088E090E00E941017BC
:10283000E12C04E021E14EE35EE06FE270E08BE02A
:1028400090E00E942D0F4AE063E070E08EE590E09A
:102850000E94661748E064E070E08FE590E00E9417
:10286000101720E14EE25EE066E070E083E690E063
:102870000E942D0FC2E6D0E021E044E163E170E068
:10288000CE010E9429162196C437D105A9F7C1E6C9
:10289000D0E021E042E164E170E0CE010E9429161F
:1028A0002196C537D105A9F742E164E170E082E6DF
:1028B00090E00E94D91642E165E270E082E690E085
:1028C0000E94D91620E042E164E170E082E690E0E7
:1028D0000E94291620E042E164E170E083E790E085
:1028E0000E94291641E16CE270E08EE590E00E94C2
:1028F00066174FE06DE270E08FE590E00E941017E0
:10290000E12C04E022E14CE15EE06FE270E082E65F
:1029100090E00E942D0FE0915101C6E0CE9FF001A2
:102920001124EA59FE4F428153816581062E000C25
:10293000770B6D5E7F4F8481082E000C990B20E091
:102940008D599F4F0E94B00EE0915101CE9FF00132
:102950001124EA59FE4F408151816581062E000CF9
:10296000770B6D5E7F4F8481082E000C990B20E061
:102970008D599F4F0E94730E40918F02509190028B
:1029800020E064E18DE10E94A71140916201509125
:10299000630120E064E380E70E94A71140918E026A
:1029A00050E04F5F5F4F20E064E389E1DF91CF911A
:1029B0000F91EF900C94A7110C942D182F923F9229
:1029C0004F925F926F927F928F929F92AF92BF923F
:1029D000CF92DF92EF92FF920F931F93CF93DF93EB
:1029E0007C016B0166246394712C00E010E0C3E06D
:1029F000D0E09AEF892E99249A942EEFA22EBB2430
:102A0000BA94842F8470282E842F8270482E842FAD
:102A10008870382E4170542E0F5F1F4F82E0680E71
:102A2000711CA60CB71C2220B1F020E0A6014C0FAF
:102A30005D1FB701600F711F85E297E00E949A1039
:102A400020E0A601400F511FB7016C0F7D1F85E2EA
:102A500097E00E949A104420B1F020E0A6014C1BA0
:102A60005D0BB701600F711F85E297E00E949A101D
:102A700020E0A601401B510BB7016C0F7D1F85E2C2
:102A800097E00E949A103320B1F020E0A601400F99
:102A9000511FB7016C1B7D0B85E297E00E949A10D5
:102AA00020E0A6014C0F5D1FB701601B710B85E292
:102AB00097E00E949A105520B1F020E0A601401B3B
:102AC000510BB7016C1B7D0B85E297E00E949A10B9
:102AD00020E0A6014C1B5D0BB701601B710B85E26A
:102AE00097E00E949A100C171D074CF4B7FC94CF86
:102AF000219782E0880E911CA80CB91C8DCFDF9124
:102B0000CF911F910F91FF90EF90DF90CF90BF90EA
:102B1000AF909F908F907F906F905F904F903F907D
:102B20002F9008957F928F929F92AF92BF92CF92F3
:102B3000DF92EF92FF920F931F93CF93DF936C017D
:102B40005B017A0180910701882309F46BC08091B1
:102B50002003882309F466C080911E0380FF05C00E
:102B60008091E00082608093E000E70110E00AEFCE
:102B700083E0982E90E4792E2AE3822E209709F4A0
:102B800048C08FB7F8949092E9009091E80095FFC3
:102B900006C09091F200272D291B922F01C090E0D2
:102BA0008FBF91110AC0015009F43CC061E070E090
:102BB00080E090E00E94EF0DE1CF292F30E0C217B6
:102BC000D3070CF49C2F8FB7F8949092E9002091D2
:102BD000E80025FF1CC0292F30E0C21BD30BF501F4
:102BE000915020F041914093F100FACFA20EB31E14
:102BF000112319F08092E80009C09091E80095FD3A
:102C000006C08092E80011E0209709F010E08FBF25
:102C1000B5CF1111B6CF5D9884E680931D031E14C5
:102C20001F0444F081E090E0F6019383828380E00A
:102C300090E001C0C701DF91CF911F910F91FF90EC
:102C4000EF90DF90CF90BF90AF909F908F907F904C
:102C50000895DF92EF92FF920F931F93CF93DF932C
:102C60007C01D22E8B01040F111DEB0177FF0EC0EA
:102C7000C0E0D0E00BC0C417D5077CF42D2DAE0109
:102C8000B70185E297E00E949A102196A8010134CD
:102C900011058CF340E450E0EECFDF91CF911F910E
:102CA0000F91FF90EF90DF9008952F923F924F92F7
:102CB0005F926F927F928F929F92AF92BF92CF92CC
:102CC000DF92EF92FF920F931F93CF93DF936C01EC
:102CD0005B01422EEE24E394F12C00E010E0C5E00D
:102CE000D0E096EF892E99249A942CEF622E7724C7
:102CF0007A94842F8170282E33243394340C4270BC
:102D0000542E0F5F1F4F82E0E80EF11C6E0C7F1CEB
:102D10002220B9F04C2F440F430D21E0B5016C1B6C
:102D20007D0BC601800F911F0E94291621E0442DC2
:102D30004E0DB501601B710BC6018C0F9D1F0E94CB
:102D400029165520B9F04C2F440F430D21E0B50151
:102D50006C1B7D0BC601801B910B0E94291621E084
:102D6000442D4E0DB501601B710BC6018C1B9D0BD4
:102D70000E9429160C171D074CF477FCC2CF21972F
:102D800082E0880E911C680C791CBBCFDF91CF913B
:102D90001F910F91FF90EF90DF90CF90BF90AF9079
:102DA0009F908F907F906F905F904F903F902F906B
:102DB00008959C01240F311D1216130684F58038E6
:102DC00091056CF5FC0197FF02C0E0E0F0E02138CE
:102DD000310514F020E830E02E1BAB014770552779
:102DE00081E090E001C0880F4A95EAF7809577FF6F
:102DF00002C0695F7F4F93E0759567959A95E1F7FB
:102E00007695762F662777956795E60FF71FEF5D26
:102E1000FC4F215020F0908198239193FACF089590
:102E2000BF92CF92DF92EF92FF920F931F93CF93B7
:102E3000DF938C01EB01B42E6C0183E0C80ED11C32
:102E40006034710520F442E1C6010E94D9167E016A
:102E5000EB0CF11CB701615071096034710520F46D
:102E600042E1C6010E94D9168AEFB80E239620E0EF
:102E70004B2DBE01C8010E94291620E04B2DBE013A
:102E8000C80147960E94291641E0BE01C6010E9472
:102E9000DE140C5E1F4F42E0BE01C8010E94DE142A
:102EA00084E0E81AF10844E0B701C8010E94DE148A
:102EB00048E0B701C601DF91CF911F910F91FF90BC
:102EC000EF90DF90CF90BF900C94DE148F929F9282
:102ED000AF92BF92CF92DF92EF92FF920F931F9328
:102EE000CF93DF936C018B01C42F7C0185E0E80E4A
:102EF000F11C460185E1880E911C5701A814B90404
:102F000051F021E04C2FB801C5010E9429168FEF26
:102F1000A81AB80AF3CFD0E02B970B5F1F4F9E0182
:102F200041E0B801C60144960E9455169E0142E058
:102F3000B801C701DF91CF911F910F91FF90EF90E2
:102F4000DF90CF90BF90AF909F908F900C945516CC
:102F50005F926F927F928F929F92AF92BF92CF9229
:102F6000DF92EF92FF920F931F93CF93DF93EC01C9
:102F70008B017A01A901461B570B57FF03C05195DE
:102F800041955109C7018C1B9D0B97FF03C091957B
:102F900081959109552453948417950714F0512C69
:102FA0000AC09E2D8F2D7901292F382F9C2F8D2F10
:102FB000E801092F182FEC16FD0654F4902F812FED
:102FC0008901292F382F9C2F8D2FE701E92EF82E0C
:102FD00037016C1A7D0A5901A01AB10AB7FE03C065
:102FE000B194A194B108630177FE03C08FEFC81AB2
:102FF000D80AD594C7940217130714F08FEF01C0B5
:1030000081E0882E880F9908EC16FD06B4F021E0C7
:10301000552019F0AE01B80102C0A801BE0185E239
:1030200097E00E949A10CA18DB08D7FE04C0080D6A
:10303000191DC60CD71C2196E7CFDF91CF911F91A8
:103040000F91FF90EF90DF90CF90BF90AF909F9047
:103050008F907F906F905F900895809121038EBD37
:10306000E2E2F3E081910DB407FEFDCF8EBD87E073
:10307000E132F807B9F70DB407FEFDCF089520E05F
:1030800081E293E0B22FB111BFEFFC010024B193B4
:10309000B193B193B1930394D1F70895809108014E
:1030A000853009F5E5EEF5E1E4918FEF80930801B5
:1030B000E13071F050F0E33089F0E430A1F4809118
:1030C00072008F7B809372000EC010926E000BC056
:1030D00080916F008D7F80936F0005C0809171009B
:1030E0008D7F80937100EBECF5E14491ECEAF5E122
:1030F0009491EDE8F5E18491882309F44DC04423CF
:10310000E1F150E0FA013197EF30F105B0F5EA5AFC
:10311000FF4F0C941C2A209180002F7707C020912C
:1031200080002F7D03C020918000277F20938000A6
:1031300024C024B52F7702C024B52F7D24BD1DC027
:10314000209190002F7707C0209190002F7D03C021
:1031500020919000277F209390000FC02091C00005
:103160002F7703C02091C0002F7D2093C00005C0A1
:103170002091C200277F2093C200E82FF0E0EE0FDD
:10318000FF1FE658FA4EA591B4918FB7F894EC91D1
:1031900090959E239C938FBF0895FC0180912003FE
:1031A000811103C08FEF9FEF08959FB7F89482E0DD
:1031B0008093E9002091F20030E01216130614F417
:1031C00021E030E02115310559F0289884E68093FC
:1031D0001F038091F10080838091F200882319F011
:1031E0009FBFC90108958BE68093E800F9CF8091D5
:1031F000430781110DC082E080933F0784E08093F4
:103200004007109242071092410781E080934307E4
:103210008FE397E00895CF93DF931F92CDB7DEB78A
:103220006983DC01ED91FC910280F381E02D41E0A6
:1032300050E0BE016F5F7F4F09950F90DF91CF91F6
:10324000089583E08093E9008091F200882319F0CB
:103250008AE38093E8000895FC018485958597FDB5
:103260000BC09FB7F89482E08093E9008091F20050
:103270009FBF90E0019608959FB7F89482E08093F5
:10328000E9008091F2009FBF90E0089540919F0770
:103290005091A00720919D0730919E074217530738
:1032A000B4F49091E8009570E1F39091E80092FDFC
:1032B00019C08093F10080919F079091A00701961B
:1032C0008F739927892B19F48EEF8093E8008091F2
:1032D0009F079091A00701969093A00780939F0766
:1032E00081E0089580E00895DF92EF92FF920F93BE
:1032F0001F93CF93DF93D82E8A017B01E40EF51E36
:10330000EB01CE15DF0571F0D7FE03C0FE018491FD
:1033100001C088810E94461921968111F2CF8FEF5A
:103320009FEF01C0C801DF91CF911F910F91FF90D6
:10333000EF90DF900895615030F02091F100FC0192
:1033400020830196F8CF289884E680931F03089580
:10335000CF93DF931F92CDB7DEB7FC0184859585AF
:1033600097FD05C02FEF3FEF358724870BC0CE01B7
:1033700001960E94CD18019719F4898190E002C04E
:103380008FEF9FEF0F90DF91CF9108950F931F93D1
:10339000CF93DF931F92CDB7DEB78C01FC018485FC
:1033A000958597FF0EC0CE0101960E94CD1801971A
:1033B00019F4298130E002C02FEF3FEFF801358783
:1033C0002487F801848595850F90DF91CF911F9117
:1033D0000F9108950F931F93CF93DF931F92CDB753
:1033E000DEB782E0898342E450E066EE75E180E872
:1033F0000E9474190E94F718DC0112960D911C911D
:1034000013970115110569F0D801ED91FC91028027
:10341000F381E02DBE016F5F7F4FC801099597FFD3
:1034200007C089810F90DF91CF911F910F9108956F
:10343000F80100851185E5CF1F920F920FB60F920C
:1034400011248F939F938091E1009091E100937FED
:103450009093E10083FF0FC01092E90091E09093F8
:10346000EB001092EC0092E39093ED001092200399
:1034700098E09093F00082FF20C093E09093E900E1
:103480009091F200992319F09AE39093E8009091BB
:103490001D03992339F090911D03915090931D03C2
:1034A000992389F190911F03992339F090911F037B
:1034B000915090931F03992341F184FF10C0809194
:1034C000E2008E7E81608093E2008091E1008F7E39
:1034D0008093E10080911E038E7E806111C080FF89
:1034E00016C08091E2008E7E80618093E200809120
:1034F000E1008E7E8093E10080911E038E7E8160CC
:1035000080931E0304C05D9ACDCF289AD6CF9F9199
:103510008F910F900FBE0F901F9018951F920F92D2
:103520000FB60F921124CF92DF92EF92FF920F937A
:103530001F932F933F934F935F936F937F938F933B
:103540009F93AF93BF93EF93FF93CF93DF93CDB749
:10355000DEB76C97DEBFCDBF1092E9008091E80026
:1035600083FFEDC168E0CE0145960E949B1982EF72
:103570008093E8008D8987FF05C09091E80090FF57
:10358000FCCF03C09EEF9093E800982F907609F04F
:10359000C6C09E892F89188D91110CC0803829F4DE
:1035A00080919C078093F10002C01092F10010926C
:1035B000F10048C1422F50E0512B913051F481115C
:1035C00041C14130510509F03DC180919C078D7F7B
:1035D0000BC0933061F4811135C14130510509F0C0
:1035E00031C180919C07826080939C072BC19530EC
:1035F00041F48091E80080FFFCCF20682093E30035
:1036000021C1963009F05FC0EB8CFC8C1092E90070
:103610001092A00710929F07123091F510929E070A
:1036200010929D070E94EA1999E0BE016F5F7F4FDB
:10363000DB01E92F1D92EA95E9F799831A8391E05E
:103640009E8390EA98879AEF998720919F073091FF
:10365000A007275F3F4F3C832B838D831092E900A7
:103660001092A00710929F07F0929E07E0929D078C
:1036700049E050E080E00E9474190E94EA19E2C01B
:10368000F0929E07E0929D070E94F718DC011296C7
:10369000ED90FC901397E114F10409F4C0C0D70138
:1036A000ED91FC910480F581E02DBE016B5E7F4FB2
:1036B000C7010995009719F00CF0C4C0C7C0F70105
:1036C000E084F184E8CF973009F4C0C0983021F449
:1036D00081E08093F100B6C0993009F0B3C08370E7
:1036E00009F0B4C0E2E3F1E081E021E036E390814B
:1036F000992361F08093E9002093EB0091919093DE
:10370000EC003093ED008F5F873089F78EE7809370
:10371000EA001092EA008F898093200393C08B8D7A
:103720009C8D1092E9001092A00710929F07909331
:103730009E0780939D07898D811156C08E899D8932
:10374000913A59F4813209F081C047E050E060E0DD
:1037500071E080E00E94741975C0913209F076C062
:10376000833289F4888D90E0982F88272F89822BC7
:10377000A0E0B0E08093090190930A01A0930B01AF
:10378000B0930C015FC0803269F48091E80082FF41
:10379000FCCF67E080E091E00E949B198BEF809363
:1037A000E80006C0823209F04DC08F89809307017E
:1037B00080919B07882319F0EEEFFAE002C0E0E069
:1037C000F8E08091000190910101A0910201B09177
:1037D0000301803B9440A105B10509F07BC08091B5
:1037E000070180FF93C076C00E94F718DC01129693
:1037F0000D911C9113970115110541F1D801ED911F
:10380000FC910190F081E02DBE016B5E7F4FC801FD
:103810000995811117C0F80100851185ECCF113091
:1038200009F44EC0133091F48F89882309F445C000
:10383000823081F440E867E08AE496E10E9417252F
:10384000882321F08EEF8093E80079C081E2809395
:10385000EB0075C0813029F440E86BE08EE396E11F
:10386000EDCF833099F70E94F718DC011296ED90A6
:10387000FC9013978E010F5F1F4F6801E114F10454
:1038800079F0D701ED91FC910680F781E02DB80128
:10389000C7010995080F111DF701E084F184EECFEF
:1038A000D8011C92F60101900020E9F73197BF0181
:1038B0006C197D0940E0C601C1CF68E276E102C023
:1038C0006CE276E16115710509F2FB01449150E06B
:1038D00080E840CF0FB6F894A89580916000886189
:1038E00080936000109260000FBEA895EE3F2AE022
:1038F000F20739F08091FE0A9091FF0A918380834C
:10390000A1CF1092FF0A1092FE0A9CCFEE3F8AE0F0
:10391000F80731F0808191819093FF0A8093FE0A2D
:1039200087E797E7918380839BE088E10FB6F8945F
:10393000A895809360000FBE9093600083CF6C9633
:103940000FB6F894DEBF0FBECDBFDF91CF91FF91D0
:10395000EF91BF91AF919F918F917F916F915F9107
:103960004F913F912F911F910F91FF90EF90DF901A
:10397000CF900F900FBE0F901F901895CF93DF93AD
:1039800000D000D01F92CDB7DEB7789484B58260A6
:1039900084BD84B5816084BD85B5826085BD85B5F3
:1039A000816085BD80916E00816080936E00109271
:1039B00081008091810082608093810080918100EC
:1039C000816080938100809180008160809380007D
:1039D000809191008260809391008091910081603C
:1039E00080939100809190008160809390008091FD
:1039F000C10084608093C1008091C1008260809387
:103A0000C1008091C10081608093C1008091C3009A
:103A100081608093C3008091C00082608093C00069
:103A20008091C20081608093C20080917A0084609E
:103A300080937A0080917A00826080937A008091EE
:103A40007A00816080937A0080917A008068809308
:103A50007A001092200310929C0710921E0380910E
:103A6000D70081608093D70080EA8093D80089B521
:103A7000806189BD89B5826089BD09B400FEFDCF32
:103A800061E070E080E090E00E94EF0D8091D8004E
:103A90008F7C80618093D8008091E000807F80934C
:103AA000E0008091E1008E7E8093E1008DE08093C4
:103AB000E200559A209AEEEFFFE7859194918B3FB3
:103AC0009C4D19F481E080939B0781EC80937C00EE
:103AD00085B1806F85B9249884B1866E84B95E9A69
:103AE0005F988AB1806D8AB9769A6E9881B3806F3B
:103AF00081BB899880B38D7080BB80E58CBD81E0EF
:103B00008DBD85E090E00E94EF0E5F9A85E090E029
:103B10000E94EF0E5E985C9808E012E08DE0F82EAF
:103B2000F00EF80184910E941C0F0F5F1F4FF012DE
:103B3000F8CF5C9A81E88093640081E0809365000F
:103B400000E014E080E00E941C0F01501109D1F741
:103B50000E94F40E87FF1FC05C9885EA0E941C0F2C
:103B60005C9A2E982F982D988091640080628093A3
:103B700064000E94110FFDCF2D980E94F40E8478EE
:103B8000843871F00E94F40E8471843131F188EC34
:103B900090E00E94EF0E0E94F40E82FDEDCF3AC03D
:103BA0000E94ED0E88EC90E00E94EF0E2F9882E0CC
:103BB00090E00E94B0258F3F29F06FEF82E090E007
:103BC0000E94B82584EF91E00E94EF0E2F9A0E9488
:103BD000F40E84788438D9F3D5CF0E94ED0E88ECAA
:103BE00090E00E94EF0E2E9882E090E00E94B025B7
:103BF000882329F060E082E090E00E94B82584EFFD
:103C000091E00E94EF0E2E9A0E94F40E847184318E
:103C1000D9F3BDCF0E94ED0E82E090E00E94B02566
:103C2000882319F00E94270F02C00E94220F2E98AD
:103C3000BEEECB2EDD24DA940E94F40E86FF04C083
:103C40002E9A2F9A2D9A41C0FCEFCF16FFEFDF0678
:103C500019F42E9A2F9806C028E1C216D10411F447
:103C60002F9A2D980E943F18EE24E39400E128E556
:103C700048E551E0B60184E190E00E942D0F0E94DA
:103C80002D188BE190E00E94EF0E30EFC3163FEF4E
:103C9000D30621F48AEF90E00E94EF0E4FEFC41A92
:103CA000D40A89E1C816D10439F68CEB92E00E945F
:103CB000EF0E0E94ED0EE0912507F091260701908E
:103CC000F081E02D85E297E0099582E390E00E9483
:103CD000EF0E0E94F40E8111F8CF80E180932C0743
:103CE000809164008E7F8093640080917A0080646C
:103CF00080937A0080917A0086FDFCCF0091780055
:103D0000109179000E94CA0D20E030E0980111273F
:103D10000027600F711F821F931F611571058105B8
:103D2000910511F00E94A725809164008160809325
:103D300064001092E8021092E90281E293E090930D
:103D4000930280939202ECE4F1E0E49180917B0095
:103D5000E3FBAA24A0F8B12CF5E0AA0CBB1CFA9551
:103D6000E1F78F7D8A2980937B00E770E064E09320
:103D70007C0080917A00806480937A0080917A0040
:103D800086FDFCCF609178008091790070E0782BFF
:103D9000072E000C880B990B6115710581059105A3
:103DA00011F00E94A72589E392E090933901809356
:103DB000380185E392E090933B0180933A0181E3DF
:103DC00092E090933D0180933C018DE292E09093CC
:103DD0003F0180933E0189E292E0909341018093FC
:103DE000400185E292E0909343018093420181E299
:103DF00092E090934501809344018DE192E090938D
:103E000047018093460189E192E0909349018093B4
:103E1000480185E192E090934B0180934A01109212
:103E2000E7021092E60281E08093EC0267E0462E02
:103E3000512C612C712C79E9272E76E0372E2FB783
:103E4000F89480914C0190914D01A0914E01B09158
:103E50004F012FBF409131075091320760913307D6
:103E60007091340720913507222341F020912D07CE
:103E7000821B809336071092350744C58417950737
:103E8000A607B70738F4481B423008F43BC50E9428
:103E9000110F38C521E02093350780932D079093AB
:103EA0002E07A0932F07B093300720912C07820F85
:103EB000911DA11DB11D8093310790933207A093EE
:103EC0003307B09334078091280790912907019612
:103ED00090932907809328070E94F40E1091E9021D
:103EE000109518231093E8028093E9029091EC0258
:103EF000923009F4C7C008F0BEC0913009F002C585
:103F00001092E1021092DF0270E17093E20222E06F
:103F10002093EC0288EE8093E0024EE155E050934E
:103F2000A00240939F0245E055E05093A2024093C7
:103F3000A10264E46093A3021092A4021092A5026D
:103F40001092A6024BEB54E05093A8024093A702B4
:103F500041E754E05093AA024093A9028EE1809376
:103F6000AB0233E03093AC023093AD0282EE80932B
:103F7000AE0244E254E05093B0024093AF0247EDEA
:103F800053E05093B2024093B10243E44093B30232
:103F90007093B4023093B5028093B60249E953E0BE
:103FA0005093B8024093B7024BE553E05093BA02E6
:103FB0004093B90249E24093BB0245E24093BC0200
:103FC0002093BD028093BE0241E153E05093C002B2
:103FD0004093BF0247EC52E05093C2024093C102AB
:103FE0006093C30246E24093C4023093C5028093BB
:103FF000C6024BEA52E05093C8024093C7024FE812
:1040000052E05093CA024093C90231E53093CB028B
:1040100037E03093CC022093CD028093CE0244E867
:1040200052E05093D0024093CF0249E752E05093C0
:10403000D2024093D1023FE23093D3024BE140934E
:10404000D4029093D5028093D6024BE552E0509370
:10405000D8024093D7024DE352E05093DA024093E6
:10406000D90293E29093DB023093DC022093DD02CD
:104070008093DE0247C4933009F438C1943009F4C8
:10408000BDC140C48091E202807F803121F0803246
:1040900009F45BC06DC08091E1028F5F8093E10203
:1040A0009091E0029A301CF49F5F9093E0028F7130
:1040B00029F48091DF028F5F8093DF0212FF06C038
:1040C00080E28093DF028093E20252C013FF50C06F
:1040D00080915001811109C00E94270F80919402A4
:1040E00090919502892B29F402C00E94220F0E9410
:1040F0004E186091500182E090E069830E94B025E3
:104100006981681721F082E090E00E94B8258091D3
:104110005001882369F130929502209294023092E6
:104120009702209296021092980281E08093990261
:1041300080E380939A0288E080939B0210929C0215
:1041400010929E0210929D0213C08091E1028F5F37
:104150008093E10280FD05C08091DF028150809351
:10416000DF028091DF02811103C083E08093EC02C3
:104170000E943F184091E6025091E7024115510517
:1041800029F021E062E084E10E94A71100E010E044
:1041900020E04FE856E068E370E0C8010E94730E2B
:1041A000085F1F4F0038110599F75EEDE52E52E0CC
:1041B000F52EF701359740815181F7016081062E78
:1041C000000C770B870103501109F801808120E072
:1041D000082E000C990B0E94B00EF7013797408112
:1041E0005181F7016081062E000C770BF801808168
:1041F00020E0082E000C990B0E94730EF7018081BD
:1042000032979081F701891714F0908305C0319798
:104210009081890FF7018083F8E0EF1AF1082EE909
:10422000E21622E0F20629F620E047E856E062E0D6
:1042300070E081E790E00E94B00E20E04FE756E08A
:1042400062E070E081E790E00E94730E0091E0026E
:10425000002E000C110B20E04DE156E0B80180E388
:1042600090E00E94B00E20E04BEB55E0B80180E3F7
:1042700090E00E94730E8091DF0280FD12C020E06A
:1042800049E855E067E270E088E290E00E94B00EF5
:1042900020E047E555E067E270E088E290E00E94A8
:1042A000730E8091500120E0882361F04FE455E0C7
:1042B00063E070E088E790E00E94B00E20E047E401
:1042C00055E00BC04FE355E063E070E088E790E015
:1042D0000E94B00E20E047E355E063E070E088E71D
:1042E00090E00E94730E0E94DC140CC38AE39DE0F0
:1042F0009093670180936601E8EBFCE0F09369011D
:10430000E093680110926A0194E090936B0126E3B8
:104310003CE030936D0120936C0124EB3BE0309343
:104320006F0120936E012EEF2093700182E0809345
:10433000710142E35BE0509373014093720140EBE3
:104340005AE05093750140937401809376018093F5
:1043500077014EE25AE050937901409378014CEA9C
:1043600059E050937B0140937A0110927C01809335
:104370007D014AE259E050937F0140937E0148EA73
:1043800058E05093810140938001209382018093F3
:10439000830126E238E0309385012093840124EAEA
:1043A00037E03093870120938601809388018093C2
:1043B000890122E237E030938B0120938A0120EAC1
:1043C00036E030938D0120938C0180938E0186E03E
:1043D00080938F011092900210928F021092E5024A
:1043E00010928E021092E302109263011092620109
:1043F00080E1809391029093EC0284C280919102BB
:10440000982F907F9032B9F1903309F414C2903113
:1044100009F078C2982F9F7019F48F5F80939102F2
:1044200042E951E022E161E080E090E0FA01E80F2A
:10443000F91F3EEF380F3B3010F0608301C010824F
:1044400001968E30910591F72150425F5F4F211107
:10445000EBCF0E9450130E94A225A30192010E945B
:10446000C625609351010E943F180E94DC1480E22F
:104470008093910247C2982F9F7019F48F5F8093A9
:1044800091028091E5028F5F8093E502082E000C77
:10449000990B40918E022EE130E0241B3109281740
:1044A00039070CF0D8C061E080E00E94C51280900E
:1044B0006501892BB1F4882D87FC8D5F882E85944A
:1044C0008594E090640102E511E0C12CD12C082C08
:1044D000000C9908AA08BB080E2C000CFF0821E06C
:1044E00004C0839480926501B4C040E050E0F801BC
:1044F000E40FF51F80818823F1F0C501B4012D83FD
:1045000049835C830E9461260E949C260E94292682
:104510006C0D7D1DFEE0F69FC001F79F900D1124EC
:10452000FC01EE56FE4F49815C81E40FF51FEE0D54
:10453000FF1D2D8122834F5F5F4F44305105B9F637
:104540003FEFC31AD30A0C5F1F4F44E0C416D104D7
:1045500061F6209162013091630100918E02F0902A
:10456000E30290E081E1EEE08E02B001112440E030
:1045700050E0A1E0FA01E60FF71FEE56FE4FE28190
:10458000E11101C0A0E04F5F5F4F4A30510591F744
:10459000AA2369F12F5F3F4F2031E7E23E0710F079
:1045A0002FE037E2F394F9E0FF1530F40F3110F407
:1045B0000F5F01C00EE1F12C182F1123B1F04EE076
:1045C000149FB001112440E050E0FA01E60FF71FFC
:1045D000EE56FE4FDF011C97AC91A2834F5F5F4FF9
:1045E0004A30510591F71150E8CF8F5F9F5F81509E
:1045F00087FFB9CF3093630120936201F092E30209
:1046000000938E02913031F480918F02909190024C
:104610000A9619C0923031F480918F0290919002E5
:10462000889611C0933039F480918F029091900256
:104630008C599F4F08C0943054F080918F02909114
:10464000900288539F4F9093900280938F020E9414
:1046500050131092E5020091E80205FF0FC060E0E0
:104660008FEF0E94C512892B29F08091640181503F
:104670008093640181E08093E4020CC006FF0AC0CD
:1046800060E081E00E94C512892BA1F38091640152
:104690008F5FEECF1091E90215FF10C08091E40208
:1046A00091E0980F9093E4028131E4F060E08FEFA5
:1046B0000E94C512892B09F02DC114C016FF10C02D
:1046C0008091E40291E0980F9093E402813154F0DC
:1046D00060E081E00E94C512892B09F01FC102C071
:1046E0001092E40214FF0BC061E080E00E94C5124A
:1046F000892B29F0809165018E5F8093650103FF0E
:1047000020C08FEF0E948A12F0906401F7FE03C070
:104710001F2D119507C0F6E0FF151CF416E01F19B8
:1047200001C010E060E0812F0E94C512892B39F092
:104730008FEF0E941E121F0D1093640102C00E9491
:1047400070120478B1F081E00E948A121091640125
:1047500017FFEAC0012F019560E0802F0E94C5126B
:10476000892B09F4E8C081E00E941E12100F1093FB
:1047700064010E943F180E949F134EEA842E41E07C
:10478000942EC12CD12C1B821A823CE2A32EB12C78
:10479000EA81FB81E80DF91D8281882349F0E12C33
:1047A00004E024E048E15EE0B601C5010E942D0F5F
:1047B0002A813B812F5F3F4F3B832A8334E0A30E46
:1047C000B11C8A819B810A9719F79EE0890E911C82
:1047D000E4E0CE0ED11CF0E4CF16D104A1F6D090C7
:1047E0009101E090900100916501002E000C110BE9
:1047F0000850110980916401082E000C990B0B964A
:104800005C01AA0CBB1CAA0CBB1C26E0E29EC001EA
:104810001124FC01EA59FE4F7F01428153812D2D65
:10482000B801C5010E94B00EF701408151812D2DC4
:10483000B801C50156CD982F9F7049F420EE31E0A4
:104840003093EB022093EA028F5F80939102809174
:10485000EA029091EB02009729F001979093EB0206
:104860008093EA020E943F180E949F1398EFC92E7E
:10487000DD24DA948CE2A82EB12CE12C04E024E0B3
:1048800048E15EE0B601C5010E942D0FF4E0AF0ED5
:10489000B11C24E5A216B10481F734E0C30ED11C8B
:1048A00040E4C416D10431F720E04AEE5DE064E153
:1048B00070E085E390E00E94B00E20E04CEB5DE0FC
:1048C00064E170E085E390E00E94730E0E94DC14C6
:1048D0008091EA029091EB02892B11F01C7091F00B
:1048E00080918F02909190022091E6023091E70230
:1048F0002817390720F49093E7028093E60281E0BD
:104900008093EC0280E090E0892B09F498CA0E9421
:10491000000095CA80916401815003C080916401B8
:104920008F5F80936401DECE17301CF006E0011B20
:1049300013CF00E011CF0E9470121BCF0F931F9373
:10494000CF93DF938C0181E090E00E94B02580FF3F
:1049500031C08AE090E00E94B0259FEF980F9E3F03
:1049600048F522E330E0D80157963C932E935697B2
:1049700028E330E059963C932E935897CBE0D0E053
:10498000D801ED91FC910190F081E02D682FC801D4
:104990000995CE010E94B0252196C131D10581F73C
:1049A0000E942D1888EE93E0DF91CF911F910F9117
:1049B0000C94EF0EDF91CF911F910F910895049702
:1049C0000C949E24EBE4F7E01382128288EE93E0CD
:1049D000A0E0B0E084839583A683B78385E191E06E
:1049E000918380838FEF9FEF95878487E1E2F7E0E3
:1049F000138212821186128620E123879087878393
:104A0000108A118A128A138A148A85E291E09183AE
:104A100080838FE291E095838483178A168A118EB2
:104A2000108E81E0828F138E848F158E0895CF9221
:104A3000DF92EF92FF920F931F93CF93DF931F921A
:104A4000CDB7DEB7182F062FE42E862F880F8E5F86
:104A500099830E94461983E00E944619F12EC12EC7
:104A60009981D92E8C2D8F19801798F4F601E7FEC5
:104A700002C0849101C080810E944619182F80E0F5
:104A80000E9446198123FFEFCF1ADF0A8111EACF76
:104A900001C081E00F90DF91CF911F910F91FF90A6
:104AA000EF90DF90CF9008958F929F92AF92BF9238
:104AB000CF92DF92EF92FF92CF93DF93EC01688168
:104AC00079818A819B81611571058105910521F4A8
:104AD00064E279ED8BE597E02DE133EF41E050E0C2
:104AE0000E94C62549015A019B01AC01A7EAB1E425
:104AF0000E94E5256B017C01ACEEB4EFA5019401A9
:104B00000E94F325DC01CB018C0D9D1DAE1DBF1D48
:104B1000B7FF03C00197A109B04888839983AA838E
:104B2000BB83BC01CD019F77DF91CF91FF90EF90C8
:104B3000DF90CF90BF90AF909F908F9008950E948C
:104B4000542508958DE091E00E94542508956093C6
:104B50000D0170930E0180930F0190931001089541
:104B6000F999FECF92BD81BDF89A992780B5089535
:104B7000262FF999FECF1FBA92BD81BD20BD0FB679
:104B8000F894FA9AF99A0FBE01960895052E97FBAC
:104B90001EF400940E94DD2557FD07D00E94F825E1
:104BA00007FC03D04EF40C94DD25509540953095CC
:104BB00021953F4F4F4F5F4F089590958095709589
:104BC00061957F4F8F4F9F4F08950E941A26A59F92
:104BD000900DB49F900DA49F800D911D11240895F8
:104BE000B7FF0C94E5250E94E525821B930B0895E1
:104BF000A1E21A2EAA1BBB1BFD010DC0AA1FBB1FE1
:104C0000EE1FFF1FA217B307E407F50720F0A21B52
:104C1000B30BE40BF50B661F771F881F991F1A94BF
:104C200069F760957095809590959B01AC01BD01E9
:104C3000CF010895A29FB001B39FC001A39F700D43
:104C4000811D1124911DB29F700D811D1124911D94
:104C500008950E9430266894B1110C941727089586
:104C60000E94E42688F09F5798F0B92F9927B751F2
:104C7000B0F0E1F0660F771F881F991F1AF0BA9500
:104C8000C9F714C0B13091F00E941627B1E0089521
:104C90000C941627672F782F8827B85F39F0B93F13
:104CA000CCF3869577956795B395D9F73EF49095B3
:104CB0008095709561957F4F8F4F9F4F0895E89431
:104CC00009C097FB3EF490958095709561957F4F54
:104CD0008F4F9F4F9923A9F0F92F96E9BB27939502
:104CE000F695879577956795B795F111F8CFFAF412
:104CF000BB0F11F460FF1BC06F5F7F4F8F4F9F4F43
:104D000016C0882311F096E911C0772321F09EE8A0
:104D1000872F762F05C0662371F096E8862F70E006
:104D200060E02AF09A95660F771F881FDAF7880FE0
:104D30009695879597F908950E94FE2690F09F37E3
:104D400048F4911116F00C94172760E070E080E8A9
:104D50009FEB089526F41B16611D711D811D0C9497
:104D6000B3260C94CE26882371F4772321F0985033
:104D7000872B762F07C0662311F499270DC0905119
:104D8000862B70E060E02AF09A95660F771F881FE7
:104D9000DAF7880F9695879597F908959F3F31F038
:104DA000915020F4879577956795B795880F911D59
:104DB0009695879597F9089557FD9058440F551F7C
:104DC00059F05F3F71F04795880F97FB991F61F08D
:104DD0009F3F79F087950895121613061406551F04
:104DE000F2CF4695F1DF08C0161617061806991F70
:104DF000F1CF869571056105089408950E94E42617
:104E0000A0F0BEE7B91788F4BB279F3860F41616E8
:104E1000B11D672F782F8827985FF7CF86957795F4
:104E20006795B11D93959639C8F30895E894BB270B
:104E300066277727CB0197F90895FA01EE0FFF1F38
:104E4000309621053105A1F16115710561F48038B5
:104E5000BFE39B0749F168949038810561F0803881
:104E6000BFEF9B0741F099234AF5FF3FE10531056C
:104E7000210519F1E8940894E795D901AA2329F4AA
:104E8000AB2FBE2FF85FD0F310C0FF5F70F4A69574
:104E9000E0F7F73950F019F0FF3A38F49F779F9315
:104EA0000DD00F9007FC9058089546F00C94AD2754
:104EB00060E070E080E89FE308954FE79F775F939D
:104EC0004F933F932F930E9421282F913F914F9111
:104ED0005F910E949D280C94752729F416F00C947C
:104EE000A7270C9416270C94AD270E94E426A8F35C
:104EF0009638A0F707F80F92E8942BE33AEA48EBCC
:104F00005FE70E94B3280F920F920F924DB75EB7E2
:104F10000F920E946928EAECF0E00E94B0274F91BE
:104F20005F91EF91FF91E595EE1FFF1F49F0FE574E
:104F3000E0684427EE0F441FFA95E1F74195550BC1
:104F40000E94E3270F9007FE0C94D727089597F946
:104F50009F6780E870E060E008959FEF80EC08951F
:104F6000DF93CF931F930F93FF92EF92DF927B011A
:104F70008C01689406C0DA2EEF010E94B028FE0171
:104F8000E894A5912591359145915591A6F3EF01AE
:104F90000E942229FE019701A801DA9469F7DF90A7
:104FA000EF90FF900F911F91CF91DF9108959B019A
:104FB000AC0160E070E080E89FE30C9477290C94EA
:104FC000A7270C94CE260E94E426D8F39923C9F390
:104FD000940F511DA3F39150504094F059F0882341
:104FE00032F0660F771F881F91505040C1F79E3FE7
:104FF00051052CF7880F911D9695879597F908957F
:105000005F3FACF0983E9CF0BB27869577956795FF
:10501000B79508F4B1609395C1F7BB0F58F711F439
:1050200060FFE8CF6F5F7F4F8F4F9F4FE3CF0C94B0
:10503000172716F00C94CE260C94AD2768940C9488
:10504000A7270E94E426A8F39923C1F3AEF3DF93C8
:10505000CF931F930F93FF92C92FDD2788232AF048
:105060002197660F771F881FDAF720E030E040E8CD
:105070005FEB9FE3883920F0803E38F021968F77F0
:105080000E940B29E2EFF0E004C00E940B29EFE13F
:10509000F1E00E94B0278B01BE01EC01FB2E6F579F
:1050A00071097595771F880B990B0E94612628E17D
:1050B00032E741E35FE30E94B028AF2D9801AE01D3
:1050C000FF900F911F91CF91DF910E9422290C94A4
:1050D000F729FA01DC01AA0FBB1F9B01AC01BF57E6
:1050E00028F4222733274427507820C0B75190F462
:1050F000AB2F0024469537952795011CA395D2F335
:10510000002071F0220F331F441FB395DAF30ED045
:105110000C940A2961307105A0E88A07B94630F479
:105120009B01AC016627772788279078309621F07D
:10513000208331834283538308950E94B0280C94C6
:10514000F7290E94E92938F00E94F02920F09523E0
:1051500011F00C94A7270C94AD2711240C94172759
:105160000E94DC2670F3959FC1F3950F50E0551F08
:10517000629FF001729FBB27F00DB11D639FAA27AC
:10518000F00DB11DAA1F649F6627B00DA11D661FFB
:10519000829F2227B00DA11D621F739FB00DA11D1C
:1051A000621F839FA00D611D221F749F3327A00DD6
:1051B000611D231F849F600D211D822F762F6A2F72
:1051C00011249F5750409AF0F1F088234AF0EE0FD7
:1051D000FF1FBB1F661F771F881F91505040A9F704
:1051E0009E3F510580F00C94A7270C9417275F3F32
:1051F000E4F3983ED4F3869577956795B795F79540
:10520000E7959F5FC1F7FE2B880F911D96958795B7
:1052100097F908955058BB27AA270E9422290C9479
:10522000F7290E94E92938F00E94F02920F039F48A
:105230009F3F19F426F40C94AD270EF4E095E7FB9C
:105240000C94A727E92F0E94DC2658F3BA176207AF
:1052500073078407950720F079F4A6F50C941627B8
:105260000EF4E0950B2EBA2FA02D0B01B901900181
:105270000C01CA01A0011124FF27591B99F0593FC5
:1052800050F4503E68F11A16F040A22F232F342F0D
:105290004427585FF3CF469537952795A795F0405B
:1052A0005395C9F77EF41F16BA0B620B730B840B70
:1052B000BAF09150A1F0FF0FBB1F661F771F881F28
:1052C000C2F70EC0BA0F621F731F841F48F4879580
:1052D00077956795B795F7959E3F08F0B0CF939572
:1052E000880F08F09927EE0F9795879508950E94EB
:1052F0008B290C94F7290E94F02958F00E94E92983
:1053000040F029F45F3F29F00C94A72751110C9429
:1053100017270C94AD270E94DC2668F39923B1F37C
:10532000552391F3951B550BBB27AA2762177307CB
:10533000840738F09F5F5F4F220F331F441FAA1F5F
:10534000A9F335D00E2E3AF0E0E832D0915050401B
:10535000E695001CCAF72BD0FE2F29D0660F771FC9
:10536000881FBB1F261737074807AB07B0E809F0AF
:10537000BB0B802DBF01FF2793585F4F3AF09E3F34
:10538000510578F00C94A7270C9417275F3FE4F39E
:10539000983ED4F3869577956795B795F7959F5F77
:1053A000C9F7880F911D9695879597F90895E1E0C3
:1053B000660F771F881FBB1F621773078407BA0722
:1053C00020F0621B730B840BBA0BEE1F88F7E0957D
:1053D000089500240A94161617061806090608955B
:1053E00000240A9412161306140605060895092EC1
:1053F0000394000C11F4882352F0BB0F40F4BF2B30
:1054000011F460FF04C06F5F7F4F8F4F9F4F08956F
:10541000AA1BBB1B51E107C0AA1FBB1FA617B707DA
:1054200010F0A61BB70B881F991F5A95A9F78095F6
:105430009095BC01CD010895EE0FFF1F0590F491EA
:10544000E02D099481E090E0F8940C94272AF894D8
:02545000FFCF8C
:1054520000E1000000000000FFFFFFFFFF0100006D
:1054620000000000000B1992152C19A819C6192169
:105472001900000000B810540B9E24FCFF0000DF4E
:085482002400C180810000003C
:00000001FF
